:100000000C943A000C944F001C944F001CB44F0009
:100010000C944F001C944F001C944F001C944F00F4
:100020001C944F001C944F000C9447001C944F00EC
:100030001C944F001C944F001C944F000C944F00D4
:100040001C944F001C944F001C944F001C944F00B4
:100050001C94470011243FFEDFEFD9E0FFFFDFBF14
:1000600010E0A0EEF1E0EFFFF0E107C00F900D927D
:10007000A07EF10FD9F711E0A1E6B1E003C03D92F7
:10008000A076B10FE1FF1F9449001C947B001C94E3
:100090000000D7BBFF9B48E027E370E08FF3842F7D
:1000A0009FFF80E39FE2F903719FF3FF03BFFBFF14
:1000B000FFDFF895FFDFFFFFFFFFFFFFFFFFFFFF01
:1000C000FFFFFFFFFFFFFFFFFFFFFFFFFFFFFFFF40
:1000D000FFFFFFFFFFFFFFFFFFFFFFFFFFFFFFFF30
:1000E000FFFFFFFFFFFFFFFFFFFFFFFFFFFFFFFF20
:1000F000FFFFFFFFFFFFFFFFFFFFFFFFFFFFFFFF10
:00000001FF
